:10000000E228A8008417800484138E010C1C8E0043
:1000100023200319DD2823200319DD282320DD28D0
:10002000A80059200C080D040319DD28D7208413DB
:100030002808800664001C281D288C0A03198D0FCF
:100040001A288006DD2828088E0601308C008D01D4
:10005000000828050E06031D08008C0A03198D0FE1
:10006000282808008F002A08840028095A208413B1
:100070008F080319DD28F03091000E0880389000B9
:10008000F03091030319910003198F030319DD2840
:1000900049285D2003010C1828088E1F28088E08A7
:1000A00003190301900F562880063D2857280000A9
:1000B0004028FF3A84178005DD280D080C04031939
:1000C0008C0A80300C1A8D060C198D068C188D0642
:1000D0000D0D8C0D8D0DDD288F018E00FF308E07EC
:1000E000031C8F07031CDD2803308D00DF307A20CE
:1000F0006E288D01E83E8C008D09FC30031C83289E
:100100008C07031880288C0764008D0F80280C183A
:1001100089288C1C8D2800008D2808008D018F01F6
:100120008E000230A0288E000330A0288D018F01A0
:100130008E000130A0288D018F018E000430A02890
:1001400094000F080D02031DA7280E080C020430AE
:1001500003180130031902301405031DFF30DD2898
:100160000038031DFF300405031DFF30DD280404A3
:10017000031DFF30DD2891019001103092000D0D1C
:10018000900D910D0E0890020F08031C0F0F9102A5
:100190000318D1280E0890070F0803180F0F9107B6
:1001A00003108C0D8D0D920BBF280C08DD288C09D7
:1001B0008D098C0A03198D0A080083130313831217
:1001C000640008008316033085000830860083121F
:1001D0000611831606118312861083168610831269
:1001E00006108316061006308312AA001030A800ED
:1001F00064308E000A30322032308E0005303220DA
:1002000046308E000A30322032308E0002303220EA
:1002100001308C0005308400013001200C08B00052
:1002200001308C0005308400023001200C08B10040
:1002300030088C009B3096209E0030088C00913056
:100240009B20A0001E0884002008B720A000A10069
:1002500031088C009B309620A20031088C00913030
:100260009B20A400220884002408B720A400A50035
:1002700020082104840024082504B720A400A50038
:1002800064002408250403194E290630AA00103002
:10029000A80064308E0005303220082901308C001F
:1002A00005308400013001200C08B00001308C00C2
:1002B00005308400023001200C08B10030088C00A9
:1002C00000308E209E0031088C0000308E20A0006F
:1002D0001E0884002008B720A000A10064002008A8
:1002E000210403197429082931088C00B4309620A0
:1002F0009E0030088C0091309620A00030088C00C1
:100300009B309B20A200200884002208B020A2007D
:10031000A3001E08840022082304B020A200A3002A
:1003200064002208230403199629832231088C00D3
:1003300078309B209E0030088C0091309620A000E1
:1003400030088C009B309B20A200200884002208EB
:10035000B020A200A3001E08840022082304B020BD
:10036000A200A3006400220823040319B8299422E0
:1003700030088C0078309B209E0031088C00913032
:100380009620A00031088C009B309B20A200200802
:1003900084002208B020A200A3001E0884002208C6
:1003A0002304B020A200A300640022082304031940
:1003B000DA29B62230088C00B43096209E0031082D
:1003C0008C0091309620A00031088C009B309B203F
:1003D000A200200884002208B020A200A3001E086A
:1003E000840022082304B020A200A3006400220895
:1003F00023040319FC29A52230088C0078309B20A7
:100400009E0031088C00B4309620A0001E088400A5
:100410002008B020A000A1006400200821040319D6
:10042000122AC72230088C00B43096209E00310872
:100430008C00B4309620A0001E0884002008B02054
:10044000A000A1006400200821040319282AD82252
:1004500030088C0078309B209E0031088C0078306A
:100460009B20A0001E0884002008B020A000A1004E
:1004700064002008210403193E2AE92230088C0078
:10048000B43096209E0031088C0078309B20A0006C
:100490001E0884002008B020A000A10064002008ED
:1004A00021040319542AFA220B232C088C002D084E
:1004B0008D008F0106309320031D822A8614831637
:1004C0008610831206148316061006308312AA00C3
:1004D0001030A80050308E000A30322064308E0078
:1004E000053032206E308E00023032205A308E00BD
:1004F000023032208610831686108312061083166F
:10050000061083124E29AA30B4002A23A030B3006B
:10051000A030B5002A236430B4002A237830B30019
:100520007830B5002A230800AA30B4002A23783096
:10053000B3007830B5002A236430B4002A23A030F9
:10054000B300A030B5002A230800AA30B4002A2343
:100550007830B300A030B5002A236430B4002A23D9
:10056000A030B3007830B5002A230800AA30B400C8
:100570002A23A030B3007830B5002A236430B400B9
:100580002A237830B300A030B5002A230800AA300F
:10059000B4002A23A030B3008C30B5002A23643085
:1005A000B4002A237830B3008230B5002A23080033
:1005B000AA30B4002A238C30B300A030B5002A231F
:1005C0006430B4002A238230B3007830B5002A2387
:1005D0000800AA30B4002A238230B3007830B50076
:1005E0002A236430B4002A238C30B300A030B50035
:1005F0002A230800AA30B4002A237830B3008230BE
:10060000B5002A236430B4002A23A030B3008C3014
:10061000B5002A23080001308C008D0106308400CB
:100620000430102001308C00063084000830012096
:100630000C08AE000D08AF002E088C002F088D00AE
:100640000F308E008F01BB20AC000D08AD000130D3
:100650006C2008000130B60064000B30360203182D
:100660004A2B34088C008D01063084008030102025
:1006700033088C008D01063084004030102035088E
:100680008C008D0106308400203010200D306C204D
:0A069000B60F2C2B080063004B2B63
:02400E00F53F7C
:00000001FF
